S024000062696E2F64656D6F70726F675F6F6C696D6578696E6F5F73746D33322E73726563F0
S315080080000050002079820008C9820008C982000849
S31508008010C9820008C9820008C98200080000000059
S31508008020000000000000000000000000C9820008EF
S31508008030C982000800000000C9820008A98C00084F
S31508008040C9820008C9820008C9820008C9820008D6
S31508008050C9820008C9820008C9820008C9820008C6
S31508008060C9820008C9820008C9820008C9820008B6
S31508008070C9820008C9820008C9820008C9820008A6
S31508008080C9820008C9820008C9820008C982000896
S31508008090C9820008C9820008C9820008C982000886
S315080080A0C9820008C9820008C9820008C982000876
S315080080B0C9820008C9820008C9820008C982000866
S315080080C0C9820008C9820008C9820008C982000856
S315080080D0C9820008C9820008C9820008C982000846
S315080080E0C9820008C9820008C98200080000000089
S315080080F00000000000000000000000000000000072
S3150800810000000000000000005FF808F1EE11AA5513
S3150800811010B5054C237833B9044B13B10448AFF3B3
S3150800812000800123237010BD3804002000000000E1
S31508008130748E000808B5034B1BB103490348AFF317
S31508008140008008BD000000003C040020748E000872
S3150800815070B50D4E0D4D761BB61006D000240134B1
S3150800816055F8043B9847A642F9D1094E094D00F047
S3150800817081FE761BB61006D00024013455F8043B60
S315080081809847A642F9D170BDB48E0008B48E00088F
S31508008190BC8E0008B48E0008024B13B1024800F0EA
S315080081A005B8704700000000B981000800230146A1
S315080081B01A46184600F01EB838B50A4C0A4D641B14
S315080081C0A4100AD004F18043013B05EB8305013C6A
S315080081D055F804399847002CF9D1BDE8384000F025
S315080081E04FBE00BFC08E0008BC8E0008704700BF97
S315080081F0704700BF2DE9F0411D4C054620689046A2
S315080082001F460E46FFF7F2FF1A4B1A68D2F8483196
S315080082101BB35A6820681F2A24DC4DB9511C023248
S31508008220596043F82260FFF7E3FF0020BDE8F081BC
S31508008230012403EB820CCCF88880D3F8881194408B
S315080082402143022DC3F88811CCF80871E6D1D3F87A
S315080082508C110C43C3F88C41E0E702F5A673C2F80B
S315080082604831D6E7FFF7C4FF4FF0FF30DEE700BF1F
S3150800827028040020A08E0008DFF834D0002103E08F
S315080082800C4B5B58435004310B480C4B42189A422E
S31508008290F6D30B4A02E0002342F8043B094B9A4204
S315080082A0F9D300F0C1FCFFF753FF00F06EFD7047ED
S315080082B000500020C08E000800000020380400206E
S315080082C03804002084040020FEE70000074AD3682B
S315080082D023F4E0631B041B0C000200F4E06018435F
S315080082E040F0BF6040F40030D060704700ED00E019
S315080082F030B4174BDB68C3F30223C3F10704042C1D
S3150800830028BF04241D1D062D01D9033B00E00023C8
S315080083104FF0FF3505FA04F421EA0401994005FAFD
S3150800832003F322EA03031943002809DB0901C9B24A
S3150800833000F1604000F5614080F8001330BC7047DA
S3150800834000F00F000901C9B2024B1954F6E700BF45
S3150800835000ED00E014ED00E00138B0F1807F0AD2AC
S31508008360064B5860064AF02182F8231000209860D0
S3150800837007221A6070470120704700BF10E000E02E
S3150800838000ED00E0042805D0054A136823F004032D
S3150800839013607047024A136843F00403136070477A
S315080083A010E000E0704708B5FFF7FCFF08BD0000C5
S315080083B0F0B482B000263546A0E0002B58D0012B39
S315080083C010D1CE680EE0694FBB4251D048D9684FEC
S315080083D0BB424DD007F58037BB4249D0A7F5801779
S315080083E0BB4245D0FF2A57D88446FF2A57D8AC0047
S315080083F0DCF800300F27A74023EA070306FA04F43F
S315080084002343CCF800304B6813F0805F75D0594B86
S315080084109C6944F001049C619B6903F00103019384
S31508008420019BAC08A71C544B53F8273005F00307EB
S31508008430BF004FF00F0C0CFA07FC23EA0C0C4F4B4D
S31508008440984232D003F58063984270D003F5806372
S3150800845098426ED003F58063984224D0042325E021
S31508008460A7F58017BB4203D007F58037BB42B9D1C1
S315080084708B687BB1012B08D044610826B2E7CE6829
S315080084800836AFE7CE680C36ACE704610826A9E7DC
S315080084900026A7E70426A5E700F1040CA5E7A5F141
S315080084A00804A400A4E7032300E00023BB4043EA32
S315080084B00C030234304F47F824304B6813F4803FDE
S315080084C039D02F4C2368134323604B6813F4003FBD
S315080084D037D02B4C6368134363604B6813F4801FD3
S315080084E035D0274CA3681343A3604B6813F4001FC9
S315080084F033D0234CE3681A43E26001350F2D32D896
S315080085000124AC400A6822409442F6D14B68122BEB
S31508008510B8D03FF658AF022BB1D07FF64EAF032B3B
S31508008520B6D0112B7FF45EAFCE6804365AE7012326
S31508008530BCE70223BAE7124C236823EA0203236046
S31508008540C3E70F4C636823EA02036360C5E70C4C74
S31508008550A36823EA0203A360C7E7094CE36823EA92
S315080085600202E260C9E702B0F0BC704700002110C1
S3150800857000003110001002400000014000080140D0
S31508008580000401400AB1016170470904016170479E
S3150800859010B504460E4B18784FF47A73B3FBF0F314
S315080085A00C4A1068B0FBF3F0FFF7D6FE68B90F2C3B
S315080085B001D901200AE0002221464FF0FF30FFF7DB
S315080085C097FE054B1C60002000E0012010BD00BF8F
S315080085D02C040020340400203004002008B5074A83
S315080085E0136843F0100313600320FFF76FFE0020A3
S315080085F0FFF7CEFF00F0D4FB002008BD00200240A4
S31508008600034A1168034B1B780B441360704700BF7D
S31508008610800400202C040020014B1868704700BF16
S315080086208004002082B0084B1B68084AA2FB03237B
S315080086305B0A00FB03F0019000BF019B5A1E0192E2
S31508008640002BF9D102B0704734040020D34D6210D4
S3150800865070B582B00446036813F0010F2CD0AB4BFB
S315080086605B6803F00C03042B1DD0A84B5B6803F072
S315080086700C03082B12D06368B3F5803F41D0002B5A
S3150800868055D103F1804303F504331A6822F4803286
S315080086901A601A6822F480221A6037E09B4B5B68DE
S315080086A013F4803FE7D0994B1B6813F4003F03D0BF
S315080086B06368002B00F0AE81236813F0020F75D0B3
S315080086C0924B5B6813F00C0F5FD0904B5B6803F01E
S315080086D00C03082B54D02369002B00F089808C4B9F
S315080086E001221A60FFF798FF0546884B1B6813F0AE
S315080086F0020F74D1FFF790FF401B0228F5D903201B
S315080087008DE1824A136843F480331360636843B388
S31508008710FFF782FF05467D4B1B6813F4003FCBD15C
S31508008720FFF77AFF401B6428F5D9032077E1B3F5F4
S31508008730A02F09D0754B1A6822F480321A601A687D
S3150800874022F480221A60E1E703F18043A3F53C3363
S315080087501A6842F480221A601A6842F480321A6053
S31508008760D4E7FFF759FF0546684B1B6813F4003F2B
S31508008770A2D0FFF751FF401B6428F5D903204EE12C
S31508008780624B5B6813F4803FA5D1604B1B6813F0FE
S31508008790020F03D02369012B40F03E815B4A136820
S315080087A023F0F803616943EAC1031360236813F0F1
S315080087B0080F32D0A369002B5BD0564B01221A60F2
S315080087C0FFF72AFF0546514B5B6A13F0020F21D1CA
S315080087D0FFF722FF401B0228F5D903201FE14B4A69
S315080087E0136823F0F803616943EAC1031360DDE700
S315080087F0474B00221A60FFF70FFF0546434B1B68DD
S3150800880013F0020FD2D0FFF707FF401B0228F5D955
S31508008810032004E10120FFF705FF236813F0040F86
S3150800882000F09880394BDB6913F0805F33D1374B02
S31508008830DA6942F08052DA61DB6903F0805301930A
S31508008840019B0125344B1B6813F4807F25D0E36810
S31508008850012B36D0002B4CD103F1804303F50433AA
S315080088601A6A22F001021A621A6A22F004021A62CD
S315080088702CE0284B00221A60FFF7CEFE0546234B54
S315080088805B6A13F0020FC8D0FFF7C6FE401B02282A
S31508008890F5D90320C3E00025D4E71F4A136843F43B
S315080088A080731360FFF7B8FE06461B4B1B6813F46C
S315080088B0807FCCD1FFF7B0FE801B6428F5D9032052
S315080088C0ADE0124A136A43F001031362E3687BB30F
S315080088D0FFF7A2FE06460D4B1B6A13F0020F38D1AE
S315080088E0FFF79AFE801B41F288339842F3D903209A
S315080088F095E0052B12D0054B1A6A22F001021A627E
S315080089001A6A22F004021A62E0E700BF0010024069
S31508008910000042428004424200700040424B1A6AFC
S3150800892042F004021A621A6A42F001021A62CDE79C
S31508008930FFF772FE06463C4B1B6A13F0020F08D07F
S31508008940FFF76AFE801B41F288339842F3D9032069
S3150800895065E0E5B9E369002B60D0334A526802F056
S315080089600C02082A5DD0022B17D0304B00221A6061
S31508008970FFF752FE04462C4B1B6813F0007F47D0C6
S31508008980FFF74AFE001B0228F5D9032047E0264ACE
S31508008990D36923F08053D361DCE7244B00221A60A5
S315080089A0FFF73AFE0546204B1B6813F0007F06D0FA
S315080089B0FFF732FE401B0228F5D903202FE0236A71
S315080089C0B3F5803F1AD018494B6823F47413226A0A
S315080089D0606A024313434B60144B01221A60FFF787
S315080089E01BFE0446104B1B6813F0007F0ED1FFF7E1
S315080089F013FE001B0228F5D9032010E00A4A536823
S31508008A0023F40033A1680B435360DCE7002006E03B
S31508008A10002004E0012002E0012000E0002002B06E
S31508008A2070BD0120FBE700BF001002406000424213
S31508008A3010B487B0164C94E80F000DF1180C0CE929
S31508008A400F00238AADF80430124B5B6803F00C0262
S31508008A50082A03D0104807B010BC7047C3F38342F6
S31508008A60624412F8102C13F4803F0CD0094B5B6853
S31508008A70C3F34043634413F8143C074800FB02F071
S31508008A80B0FBF3F0E7E7054800FB02F0E3E700BFB9
S31508008A908C8E00080010024000127A0000093D0082
S31508008AA05A4B1B6803F007038B420BD2574A1368CD
S31508008AB023F007030B431360136803F007038B4285
S31508008AC040F09D8070B5036813F0020F06D0504A37
S31508008AD0536823F0F0038468234353600D46044625
S31508008AE0036813F0010F52D04368012B23D0022BE1
S31508008AF028D0474A126812F0020F00F082804449D3
S31508008B004A6822F0030213434B60FFF785FD0646C9
S31508008B106368012B1DD0022B2AD03D4B5B6813F0EE
S31508008B200C0F34D0FFF778FD801B41F2883398424A
S31508008B30F3D9032062E0364A126812F4003FDED108
S31508008B4001205BE0324A126812F0007FD7D101207B
S31508008B5054E02F4B5B6803F00C03042B17D0FFF788
S31508008B605BFD801B41F288339842F2D9032045E029
S31508008B70274B5B6803F00C03082B08D0FFF74CFD66
S31508008B80801B41F288339842F2D9032036E01F4B06
S31508008B901B6803F00703AB420AD91C4A136823F083
S31508008BA007032B431360136803F00703AB422AD16C
S31508008BB0236813F0040F06D0154A536823F4E063BC
S31508008BC0E1680B435360236813F0080F07D0104A77
S31508008BD0536823F46053216943EAC1035360FFF7DE
S31508008BE027FF0B4B5B68C3F303130A4AD35CD840D1
S31508008BF0094B18600020FFF7CBFC002070BD012050
S31508008C0070470120FAE70120F8E700BF002002407C
S31508008C1000100240A48E000834040020014B186896
S31508008C20704700BF340400200F4B1A6842F0010257
S31508008C301A6059680D4A0A405A601A6822F0847206
S31508008C4022F480321A601A6822F480221A605A685E
S31508008C5022F4FE025A604FF41F029A60044B4FF04A
S31508008C6000629A60704700BF001002400000FFF8DB
S31508008C7000ED00E008B5FFF7D1FF084BA3FB003075
S31508008C808009FFF769FB0420FFF77CFB00221146E9
S31508008C904FF0FF30FFF72CFB08BD00BFD34D621025
S31508008CA008B5FFF7B9FC08BD08B5FFF7A9FCFFF73B
S31508008CB07AFB08BD08B5002220210248FFF762FCAE
S31508008CC008BD00BF0008014010B5FFF7E9FF0E4BCD
S31508008CD01B68C31AB3F5FA7F0CD304460B4B1B78F3
S31508008CE04BB90122094B1A7020210948FFF74AFCA3
S31508008CF0054B1C6010BD0022044B1A702021044845
S31508008D00FFF740FCF4E700BF580400205404002095
S31508008D1000080140014A024B9A607047008000082B
S31508008D2000ED00E000B591B0012206924FF48033C1
S31508008D300793002108910A9202220D920E934FF48E
S31508008D40E0130F9306A8FFF783FC00B1FEE70F2395
S31508008D50019302210291002303934FF48062049247
S31508008D60059301A8FFF79CFE00B1FEE711B05DF878
S31508008D7004FB08B5FFF7CEFFFFF730FCFFF7D2FF7D
S31508008D80FFF778FFFFF796FF08BD08B5FFF7F1FF75
S31508008D9000F06EF8FFF798FF00F06BF8FAE70000AE
S31508008DA000B589B0304B9A6942F001029A619A6916
S31508008DB002F001020092009ADA6942F08052DA6102
S31508008DC0DA6902F080520192019A9A6942F0040225
S31508008DD09A619A6902F004020292029A9A6942F02A
S31508008DE008029A619B6903F008030393039B032017
S31508008DF0FFF76CFA002211466FF00B00FFF778FABE
S31508008E00002211466FF00A00FFF772FA0022114697
S31508008E106FF00900FFF76CFA002211466FF00400A4
S31508008E20FFF766FA002211466FF00300FFF760FAB3
S31508008E30002211466FF00100FFF75AFA0022114688
S31508008E404FF0FF30FFF754FA2023049301230593CC
S31508008E50002306930223079304A90448FFF7A8FAF8
S31508008E6009B05DF804FB00BF00100240000801408D
S31508008E7070477047F8B500BFF8BC08BC9E467047F7
S31108008E80F8B500BFF8BC08BC9E46704759
S31508008E8C02030405060708090A0B0C0D0E0F101031
S31508008E9C0102000000000020000000000000000095
S30D08008EAC010203040607080988
S30D08008EB49981000835810008C8
S30908008EBC118100080A
S31508008EC000000000EC02002054030020BC03002030
S31508008ED00000000000000000000000000000000084
S31508008EE00000000000000000000000000000000074
S31508008EF00000000000000000000000000000000064
S31508008F000000000000000000000000000000000053
S31508008F100000000000000000000000000000000043
S31508008F200000000000000000000000000000000033
S31508008F300000000000000000000000000000000023
S31508008F400000000000000000000000000000000013
S31508008F500000000000000000000000000000000003
S31508008F6000000000000000000100000000000000F2
S31508008F700E33CDAB34126DE6ECDE05000B000000B7
S31508008F8000000000000000000000000000000000D3
S31508008F9000000000000000000000000000000000C3
S31508008FA000000000000000000000000000000000B3
S31508008FB000000000000000000000000000000000A3
S315080092E000000000000000005C04002001000000EF
S30D080092F01000000000A24A0468
S70508008279F7
